:020000020000FC
:1000000008C02CC01895189537C059C01895189578
:1000100018959FEF98BB95E093BF98E090BF90E450
:100020009BBF96E099BF2224332744279BE097BBD0
:10003000C19AC39AC0985527652F252F90E395BF85
:10004000789400000000F8942530D1F79FEF98BB1A
:10005000789488956627262F69BFDBCF112059F445
:100060008FEF182E88278FBD682F282F523011F45C
:1000700054E0189555271895889481E0380F08F4B6
:1000800043954330D9F45395513011F4C19814C0BD
:10009000523021F4C09AC19AC3980EC0533051F027
:1000A000553021F4C09AC198C39A06C0573021F444
:1000B000C098C19A5A9511243327442718956A95F8
:0800C00011F471E0270F1895FF
:00000001FF
